:102D8100000A0014000500320032000A0005000AA2
:022D9100C3502D
:10278800C10B4101640101BA01011500C10AC10070
:102798000108FF4100000041014100011D00C10383
:0C27A800C182C108010B00011C00C1012E
:101EAD00E4F523F524F5A0F590F5D81212789000FD
:101EBD00007403F0121FE1122B9A300926C2097823
:101ECD006AE6600B16E6B40106200503122C0BE53D
:101EDD005FD39400400DD55F0A122DC37F0A7E009B
:101EED001217F5789FE6D394034050E4F6122DE2D5
:101EFD001223DAE4F51BE51B25E024A8F8E6FE081D
:101F0D00E6FF900165EEF0A3EFF04E6025E024FFB3
:101F1D00F0900165E034FFF0E0FEA3E0FFE51B2546
:101F2D00E024A8F8A60608A607EF4E7005AF1B1211
:101F3D002D6F051BE51BC3940940BBE5157002C150
:101F4D00C71515740C2515F8E614601E14602214BF
:101F5D00607B240370E50524E524C3940A4005E461
:101F6D00F524B204E4FDFCFF805EE4FDFC7F0180FE
:101F7D0057E5587003122B9A300E21C20EE4F5234B
:101F8D00900264E0FF12000040397F057E001217B9
:101F9D00F50523E523C3940540E68027300D21C2C6
:101FAD000DE4F523900262E0FF12000040157F055D
:101FBD007E001217F50523E523C3940540E6800343
:101FCD00122CD7E4FDFC7F02122BD6E1487F0312C1
:041FDD002BD3E148D9
:10127800E4F580122D939001B7741EF0E490029665
:10128800F0900296E0FFC394205052EF244EFF7B6B
:10129800017A027998E4F5321225A040119002965D
:1012A800E024F9F582E43401F583E4F08027D39053
:1012B8000299E09405900298E094004004E4F0A3B9
:1012C800F0900299E0FF900296E024F9F582E43468
:1012D80001F583EFF0900296E004F080A47B017A98
:1012E800027997E4F5337F0F1226FA4006900297A9
:1012F8007401F0900297E0B4010B75878090026347
:101308007403F08009E4F5879002637406F0758031
:10131800FF759850758921758DFD758BFD758A044B
:10132800758CF7D28ED28CD2A943BF021229FDD276
:10133800AFD2AC750A01122DE21217F1122DE2128A
:1013480017F1122DE21217F1122DE21217F1122DD8
:10135800E21217F1122DE2E4F50A900296F09002DB
:1013680096E0FFC394A0501B75F002EFA42401F58A
:1013780082E5F03400F583E4F0A3F0900296E004EF
:10138800F080DBE4900296F0900296E0FFC39408A8
:10139800500B74A02FF8E4F6E004F080EBE4900220
:1013A80096F0900296E0FFC39409500FEF25E024D1
:1013B800A8F8E4F608F6E004F080E7E4FBFDFC7F1B
:1013C800631228FBE4900285F07B017A017962F5CB
:1013D800337F0D1226FA40069001627480F07B017B
:1013E8007A017964E4F5337F0C1226FA400AE4FBAB
:1013F8007D01FC7F0C1228FB900164E0700FFB7DDF
:1014080001FC7F0C1228FB9001647401F0E4FB7D61
:101418000DFC7F051228FBE4FB7D16FC7F071228D4
:10142800FB7B017A007900E4F5337F081226FAE4A1
:10143800FDFCFF122BD67F02122BD3900164E064CF
:1014480002703BFDFC7F04122BD6E4900296F090CC
:101458000296E0FFC394105018EF25E02442F5826D
:10146800E43401F583E4F0A3F0900296E004F08000
:10147800DE900285E030E704D2068002C206E4FD71
:10148800FC7F08122BD6E4900296F0900296E0FFBB
:10149800C39420501474D92FF582E43401F583E401
:0914A800F0900296E004F080E2ED
:0114B1002218
:03000B000229596E
:10295900C0E0C0F0C083C082C0D075D000C000C044
:1029690001C002C003C004C005C006C007758A04BF
:10297900758CF7789F06D2097580FF78BA06E6D379
:10298900940540027601122800D007D006D005D060
:1029990004D003D002D001D000D0D0D082D083D0CF
:0429A900F0D0E03258
:102D6F00E515C39409500AAE150515740C2EF8A677
:022D7F00072229
:032BD300E4FDFC22
:102BD6008C258D26E5264525701FEF25E02481F5F9
:102BE60082E4342DF583E493FC740193FDEF25E034
:102BF60024A8F8A60408A60522EF25E024A8F8A62E
:052C06002508A62622AE
:101FE100900000E0FF7006439B4075A303EFC3948C
:0E1FF100014002D20AEFC394034002D2002244
:102CD700E558B40107D212E4FF0224C7E558B4024D
:0D2CE70003020F1CE558B403031222D4228F
:1023DA00900164E070123004055317FE800343171E
:1023EA000130031D801680193004055317FE80033F
:1023FA00431701E509D39400400715095317FD80D7
:10240A0003431702E4FF75F002EFA42431F582E5D5
:10241A00F03400F583E0FCA3E0D394F4EC9401E5F6
:10242A0016400513F5168006C3134480F5160FBF30
:10243A0008D4E4FF75F002EFA42401F582E5F03434
:10244A0000F583E0FCA3E0D394F4EC9401E5184092
:10245A000513F5188006C3134480F5180FBF08D476
:10246A00E4FF75F002EFA42411F582E5F03400F5DB
:10247A0083E0FCA3E0D394F4EC9401E5194005133E
:10248A00F5198006C3134480F5190FBF08D4E4FF79
:10249A0075F002EFA42421F582E5F03400F583E01B
:1024AA00FCA3E0D394F4EC9401E51A400513F51A61
:0C24BA008006C3134480F51A0FBF08D43D
:0124C60022F3
:1028000078BAE624FE602414603814604C146060CA
:1028100024047072C2A0C2A1C2A5C2A2E50A6005CA
:10282000E4F5808003851680D2A622C2A6C2A1C28A
:10283000A5C2A2E50A6005E4F5808003851780D271
:10284000A022C2A6C2A0C2A5C2A2E50A6005E4F504
:10285000808003851880D2A122C2A6C2A0C2A1C2D4
:10286000A2E50A6005E4F5808003851980D2A522DF
:10287000C2A6C2A0C2A1C2A5E50A6005E4F5808097
:0728800003851A80D2A22299
:042DE200759FA72210
:0417F1007F507EC3E4
:0B17F500EF1FAC0670011E4C70F622C6
:1014B20000C1814001C0804101C0804100C1814022
:1014C20001C0804100C1814000C1814001C0804112
:1014D20001C0804100C1814000C1814001C0804102
:1014E20000C1814001C0804101C0804100C18140F2
:1014F20001C0804100C1814000C1814001C08041E2
:1015020000C1814001C0804101C0804100C18140D1
:1015120000C1814001C0804101C0804100C18140C1
:1015220001C0804100C1814000C1814001C08041B1
:1015320001C0804100C1814000C1814001C08041A1
:1015420000C1814001C0804101C0804100C1814091
:1015520000C1814001C0804101C0804100C1814081
:1015620001C0804100C1814000C1814001C0804171
:1015720000C1814001C0804101C0804100C1814061
:1015820001C0804100C1814000C1814001C0804151
:1015920001C0804100C1814000C1814001C0804141
:1015A20000C1814001C0804101C0804100C1814031
:1015B20000C0C101C30302C2C60607C705C5C404F1
:1015C200CC0C0DCD0FCFCE0E0ACACB0BC90908C861
:1015D200D81819D91BDBDA1A1EDEDF1FDD1D1CDC51
:1015E20014D4D515D71716D6D21213D311D1D010C1
:1015F200F03031F133F3F23236F6F737F53534F4B1
:101602003CFCFD3DFF3F3EFEFA3A3BFB39F9F83820
:1016120028E8E929EB2B2AEAEE2E2FEF2DEDEC2C10
:10162200E42425E527E7E62622E2E323E12120E080
:10163200A06061A163A3A26266A6A767A56564A470
:101642006CACAD6DAF6F6EAEAA6A6BAB69A9A868E0
:1016520078B8B979BB7B7ABABE7E7FBF7DBDBC7CD0
:10166200B47475B577B7B67672B2B373B17170B040
:101672005090915193535292965657975595945430
:101682009C5C5D9D5F9F9E5E5A9A9B5B99595898A0
:10169200884849894B8B8A4A4E8E8F4F8D4D4C8C90
:1016A2004484854587474686824243834181804000
:1027B40041026308016800C10EC10D01620002609C
:0627C400000A025D000A9C
:1029FD00C292E47868F6786AF6FB7A00796B7F0606
:102A0D007EEF122DB708E6FFF46003EF70167B0022
:102A1D007A00796BE4F5337F061226FA4013786B52
:102A2D0076FE8002786BE6FD7C00E4FB7F061228C3
:0E2A3D00FB786BE66003B4FF04786B76FE2234
:0A2DC300C292E47868F6786AF622FE
:052DDD00C20CD292229D
:030023000226575B
:10265700C0E0C083C082C0D075D000C000C005C034
:10266700063098797868E6C394325007E606246DF9
:10267700F8A699C298900263E0F55F7868E6FD6472
:10268700077034786EE6FE6403600DEEB4060280D0
:1026970007EEB4100B200F089002617408F0804415
:1026A700EEB4100B7873E62409900261F080359040
:1026B70002617432F0802D900261E0B5050B755F01
:1026C70000786A7606D20F801B7868E6B40315781F
:1026D7006EE6B4190F9002617406F0800730990412
:1026E700C299D20CD006D005D000D0D0D082D083EA
:0326F700D0E032FE
:102C0B00786FE6FE08E67C002400F526EC3EF52501
:102C1B00AF26FE121D2D5017750905122DDD122D35
:102C2B00CDAF26AE251208EDAF26AE25120C6002F5
:022C3B002DC3A7
:041D2D008E278F2846
:101D3100900261E07868666002C322786DE6FFF484
:101D4100600DEF786B666007786DE66002C32278FC
:101D51006EE664196002A1DBFB7A00796D7D0412E5
:101D61002A938E298F2A7871E6FE08E67C002400EA
:101D7100FFEC3EFEEF652A7003EE65296002C32287
:101D81007870E6FF18E6FEC39F40028002AF067836
:101D910070E6FDEEC39D400518E6FE8002AE0578B3
:101DA1006BE6FDC39F4005EDD39E4002C322789FA1
:101DB100E6FF7E00122B50122B197C007D141206B7
:101DC100518D2BE4F52CE52CC3952B500B7F647EB4
:101DD100001217F5052C80EED322786EE6FF64031E
:101DE100600CEF64066007EF64106002C322786E36
:101DF100E6FF6406703BD3E5289408E5279400507C
:101E0100307870E6FEC394025009900285E030E01C
:101E110020C322EEC394045009900285E030E11101
:101E2100C3227870E6B40809900285E030E202C36B
:101E310022E528640A4527703CEFB4030E122B19E2
:101E41007C007D05120651786CA605786CE664016C
:101E51006002C322122B197C007D141206518D2BB6
:101E6100E4F52CE52CC3952B500B7F647E001217F3
:101E7100F5052C80EE7B007A00796D900261E024FB
:101E8100FEFD122A938E298F2A900261E0FD246BB8
:101E9100F8E6FE746C2DF8E67C002400FFEC3EFEB3
:0B1EA100EFB52A06EEB52902D322C3DC
:011EAC002213
:040C60008E278F2824
:100C6400E4F52DC212786EE6FFB4061DE4F52D748A
:100C74006D252DF8E6F599C20C300CFD122DE20518
:100C84002DE52DC3940840E722EF64036002C1837D
:100C94007872E6F52B786DE6F52CF599122CF77839
:100CA4006EE6F52C300CFD122CF4E52B25E0F52C2A
:100CB400300CFD122CF4E52DC3952B4002C1667E49
:100CC40000E528252DFFEE3527FEC3EF9464EE944E
:100CD40000505DE52D2528FF7B007A007929E4F595
:100CE400321225A04005E4F529F52A7E00E52825E1
:100CF4002DFFEE3527FEC3EF946EEE94004005E41D
:100D0400F52C8004E529F52C300CFD122CF47E0022
:100D1400E528252DFFEE3527FEC3EF946EEE9400F3
:100D24004005752C018004E52AF52C300CFDC15FCB
:100D34007E00E528252DFFEE3527FEEF64634E7017
:100D440013F52C300CFD122CF4900285E0F52C30B8
:100D54000CFDC15F7E00E528252DFFEE3527FEEF53
:100D6400249CFDEE34FFFCD3ED941FEC9400503F23
:100D7400EF25E0FFEE33FE74AF2FF58274003EF5ED
:100D840083E0F52C300CFD122CF47E00E528252D93
:100D9400FFEE3527FEEF25E0FFEE33FE74AF2FF5AF
:100DA4008274003EF583A3E0F52C300CFDC15F7E18
:100DB40000E528252DFFEE3527FEEF249CFDEE34BB
:100DC400FFFCC3ED9480EC9400503FEF25E0FFEE70
:100DD40033FE74392FF58274FF3EF583E0F52C3031
:100DE4000CFD122CF47E00E528252DFFEE3527FEA0
:100DF400EF25E0FFEE33FE74392FF58274FF3EF5E4
:100E040083A3E0F52C300CFD8051AF2D7E00E52846
:100E1400252DCFEE3527CF249CCF34FFFEC3EF948E
:100E2400A0EE94005026E4F52C300CFD122CF47E38
:100E340000E528252DFFEE3527FE74152FF5827465
:100E4400013EF583E0F52C300CFD800FE4F52C30E9
:100E54000CFD122CF4752C01300CFD122CF4052D14
:100E640081BAC212300CFD7867E6F599C20C300CD9
:100E7400FD7869E6F599C20C300C02E11B80F97823
:100E84006EE664107038F52D746D252DF8E6F52C9A
:100E9400F599C20C300CFDAF2C122CFB122DE2057F
:100EA4002DE52DC3940640E07867E6F599C20C3031
:100EB4000CFD7869E6F599C20C200C5B80FB786E1A
:100EC400E66419705218E6F52CF599C20C300CFD45
:100ED400AF2C122CFB122DE2786EE6F52CF599C29C
:100EE4000C300CFDAF2C122CFB122DE2786BE6F5C6
:100EF4002CF599C20C300CFDAF2C122CFB122DE2F8
:100F04007867E6F599C20C300CFD7869E6F599C26C
:070F14000C300CFD122DE270
:010F1B0022B3
:0408ED008E278F289B
:1008F100752D01E4F52E786EE6640660026184C30D
:10090100E5289464E5279400400241BF7870E6949D
:100911000150217872E6FD7C00E4FBFF1228FB7890
:1009210071E6FD7C00E4FB7F011228FB900285E06B
:10093100440180287870E6D39403502A7872E6FD4A
:100941007C00E4FB7F021228FB7871E6FD7C00E469
:10095100FB7F031228FB900285E04402F0FD7C003E
:10096100E4FB7F63617F7870E66408702E08E6FE21
:1009710008E67C002400FDEC3EFCE4FB7F08122825
:10098100FB900285E04404F0FD7C00E4FB7F6312F0
:1009910028FB7872E6900000F081187870E6B409BF
:1009A1001B08E6FE08E67C002400FDEC3EFCE4FBAF
:1009B1007F091228FB7872E6F55881187870E6FFF6
:1009C100B4060A7872E6FD7C00E4FB807B7870E671
:1009D100FFB40D1FC00708E6FE08E67C002400FDF9
:1009E100EC3EFCD007E4FB1228FB7872E690016232
:1009F100F081187870E6FFB40C1B7872E6FD7C007C
:100A0100E4FB1228FB7872E6900164F06002811821
:100A1100750A0181187870E6FFB410127872E6FD4C
:100A21007C00E4FB1228FB7872E6F52D81187870C2
:100A3100E6640A7027786CE66401600281187872B6
:100A4100E6FD7C00E4FB7F061228FB7872E6786BFA
:100A5100F67D067CEFE4FF122C788118E528640FFF
:100A6100452770197870E6FF7872E6FD7C00E4FB9B
:100A71001228FB7872E6B40102801F8028E5286401
:100A8100144527702B7870E6FF7872E6FD7C00E450
:100A9100FB1228FB7872E6B4010B75878090026324
:100AA1007403F08118E4F5879002637406F08118ED
:100AB1007870E6FF7872E6FD7C00E4FB617FC3E5B8
:100AC10028942CE527940140028118786FE6FE08EE
:100AD100E67C002400FFEC3ECF249CF528EF34FF98
:100AE100F527C3E5289420E52794004043D3E52862
:100AF100947FE5279400503808E6FE08E62400F5C7
:100B01002AEC3EF529D3E52A94FFE52964809480F7
:100B110040028118E52825E0FFE52733FE74012F07
:100B2100F58274003EF583E529F0A3E52AF08118EA
:100B3100C3E5289480E527940050028118D3E52865
:100B4100949FE527940040028118E5282480F52C24
:100B51007872E6FFC394064002811874F9252CF5DA
:100B610082E43401F583EFF0E52C244EFF74F9257E
:100B71002CF582E43401F583E0FD7C00E4FB1228CE
:100B8100FB8118786EE66410600281187872E6F9CC
:100B9100786FE6FE08E67C002400FFEC3ECF249C43
:100BA100F528EF34FFF527E4FDE9FFC3ED9FEC9451
:100BB100005064122DE2E5282DFFE5273CFEC3EF2E
:100BC1009420EE94005008EF947FEE94005041AFD2
:100BD10005EF25E0FB2474F8E6FE74752BF8E67A40
:100BE100002400F52AEA3EF529D3E52A94FFE529F8
:100BF10064809480501AE52825E0FFE52733FE74D0
:100C0100012FF58274003EF583E529F0A3E52AF072
:100C11000DBD00010C8092E52D647F70357F771248
:100C21002D11E4F52B7B007A00792CE4F533AF2B01
:100C31001226FA500DE4252BFDE434EEFCAF2C1204
:100C41002C78052BE52BD3941040DAC2AF759F8029
:0E0C510080FEE52DB4FF07C2AF759F8080FEC8
:010C5F002272
:092DCD00786976FF786776FF2231
:072CF400852C99C20CAF2CE6
:102CFB007867E66FFF9014B2937869667967F7EFA0
:052D0B009015B293F6E3
:012D100022A0
:082A93008B2D8A2E892F8D3056
:102A9B007531007532FF7DFFAF301530EF6026AB1F
:102AAB002D052FE52FAA2E7002052E14F91205E71E
:102ABB006532FF9014B2936D753100F532EF9015BE
:0A2ACB00B293FD80D3E532FEEDFF6B
:012AD50022DE
:022D5B00000076
:0727CA004101B800015800B5
:102B9A00E4F525755801D212FF1224C75003752592
:102BAA0001755802120F1C5003752502755803123D
:102BBA002AD6EFD3940040028F25852558E558FD83
:092BCA007C00E4FB7F090228FBFA
:100F1C001229AD9001B8E0FF139290EFA2E19291EB
:100F2C00A2E292937006C294D2958008EFB410049A
:100F3C00D294C295EFC39408500280149001B8E08B
:100F4C00C39410500280169001B8E0C3941850045A
:100F5C007FB5800B9001B8E0C3942050057FB1128F
:100F6C002C96122887EF4E600280287F017E00129B
:100F7C0017F5122A518E568F57122C3D40028013B2
:100F8C007F017E001217F5122A518E268F27122C04
:100F9C003D4005122DD6C3227F017E001217F5129B
:100FAC002A518E288F29122DD6E5572527FFE55675
:100FBC0035265403F52A8F2B9001B8E0700EE529E5
:100FCC00B52B20E528B52A1B7D1F8010E529B52BF4
:100FDC0012E528B52A0D9001B8E014FDAF27AE2616
:100FEC00121B8E9001B8E004F0E0D3941F4002E491
:020FFC00F0D330
:010FFE0022D0
:102AD6001229AD7FB9122C96122887EF4E60061286
:102AE6002DD67F00227F017E001217F5122A518F04
:102AF60026122C3D7F017E001217F5122A518F27D0
:102B0600E5266227122DD6E52770028003E4F52616
:022B1600AF26E8
:012B1800229A
:102D4700E5596FFF9014B293655AF559EF9015B294
:032D570093F55A97
:012D5A002256
:1022D4007559FF755AFF1229AD7FB7122C96122833
:1022E40087EF4E600280167F017E001217F5900181
:1022F400B8E0FF122C96122887EF4E6003022DD609
:102304007F017E001217F5122A518F52122C3D7F45
:10231400017E001217F5855225122A518F53122C73
:102324003D7F017E001217F5E5536225122A518F75
:1023340054122C3D7F017E001217F5E554622512DC
:102344002A518F55122C3D7F017E001217F5E55559
:102354006225122A51AD079001B8E025E0FFE4336D
:10236400FE74672FF58274013EF583EDF0122C3D67
:102374007F017E001217F59001B8E025E0FFE433F9
:10238400FE74672FF5827401122A4BAD079001B8D1
:10239400E025E0FFE433FE74682FF58274013EF516
:1023A40083EDF0122C3D7F017E001217F59001B8E9
:1023B400E025E0FFE433FE74682FF5827401122AED
:1023C4004BEF6225122DD69001B8E004F0E0D394CF
:0523D400074002E4F0E7
:0123D90022E1
:0224C7008F265E
:1024C90078277C007D007BFF7A2D795B7E007F1465
:1024D9001205C1C290C291C2931229AD3012047F74
:1024E900B180052012057FB2122C967F017E001261
:1024F90017F5122887EF4E600280167F017E0012C1
:1025090017F5122A518E278F28753B01122C3D4051
:1025190005122DD6C3227F017E001217F5E53B1364
:102529009290E53BA2E19291A2E29293122A51E59F
:102539003B25E02427F8A60608A607053BE53BD37B
:10254900940940C8122DD6E528252ACFE527352933
:10255900CF252CCF352BCF252ECF352DCF2530CFDD
:10256900352FCF2532CF3531CF2534CF3533CF2550
:1025790036CF3535CF2538CF35375403FEE53AB553
:102589000713E539B5060E7B007A007927852640C1
:062599007D081219CBD3EE
:01259F002219
:1029AD00C2B47F017E001217F5D2B5D2B47F027E7C
:1029BD00001217F5C2B57F057E001217F5C2B47F60
:1029CD00027E001217F5E558B402028005E558B4F1
:1029DD00031DD2B5D2B47F027E001217F5C2B57FAA
:1029ED00057E001217F5C2B47F027E001217F52284
:102C3D00E4FFFE20B50D0FBF00010EEF64644E7072
:102C4D00F2C322D2B57F017E001217F5D2B4C2B500
:0C2C5D007F017E001217F5D2B5C2B4D37F
:012C69002248
:022C9600AD0788
:102C98007B08ED3392B5D2B47F017E001217F5C2DE
:0E2CA800B47F017E001217F5ED25E0FDDBE4A0
:012CB60022FB
:062A4B003EF583E0622568
:102A5100E4FBFAE558B403047D0880027D0AE4F939
:102A6100E9C39D5028D2B47F017E001217F5D2B57B
:102A7100EB25E0FFEA33FEA2B5E433FBEEFAEF4BC0
:102A8100FBC2B47F017E001217F50980D3AE02AFFD
:012A91000341
:012A92002221
:072DD600C2B5D2B4D2B52250
:10288700E4F53CF53DE55864017018D2B5D2B4FAC9
:10289700FB20B50280460BBB00010AEB640A4A70B5
:1028A700F0804AE5586402701DFAFB20B50BD2B4DC
:1028B7007F017E001217F580230BBB00010AEB6432
:1028C700324A70E78027E55864037027FAFBD2B5D0
:1028D70020B50FD2B47F017E001217F5C2B4E4FE13
:1028E700FF220BBB00010AEB64324A70E1C2B47EDF
:0328F700007F015E
:0128FA0022BB
:061B8E008E2C8F2D8D2E20
:101B940075F002E52EA42401F582E5F03400F58306
:101BA400E0FEA3E0FFC3E52D9FFFE52C9EFE122D72
:101BB400A5D3EF9464EE64809480404974D9252EB3
:101BC400F582E43401F583E004F074D9252EF5821E
:101BD400E43401F583E0D3648094825002818774F5
:101BE400D9252EF582E43401F583E4F075F002E59D
:101BF4002EA42401F582E5F03400F583E52CF0A34E
:101C0400E52DF0807E74D9252EF582E43401F58328
:101C1400E4F075F002E52EA42401F582E5F0340029
:101C2400F583E0FEA3E0FFE4FCFD7B02FAF9F81281
:101C34000757C004C005C006C007AE2CAF2DE4FC96
:101C4400FD7B08FAF9F8120757D003D002D001D06F
:101C540000EB2FFFEA3EFEE93DFDE83CFCE47B0A95
:101C6400FAF9F81207E28F328E318D308C2F75F02D
:101C740002E52EA42401F582E5F03400F583EEF0AC
:101C8400A3EFF075F002E52EA42401F582E5F0340B
:101C940000F583E0FCA3E0FD74F9252EF582E4341D
:101CA40001F583E0FF7B807A00122000E52E25E019
:101CB4002477F582E43401F583EEF0A3EFF075F0B8
:101CC40002E52EA42401F582E5F03400F583E0FE5C
:101CD400A3E0D39400EE9404401675F002E52EA41C
:101CE4002401F582E5F03400F5837404F0A3E4F0F4
:101CF40075F002E52EA42401F582E5F03400F583A5
:101D0400E0FEA3E0FFE4FCFD7B607AEAF9F8C3128D
:101D14000882501475F002E52EA42401F582E5F042
:081D24003400F583E4F0A3F0A4
:011D2C002294
:0819CB008B3C8A3D893E8D3FF3
:1019D300E4F543E543C3953F4002618DAB3CAA3D2B
:1019E300A93EE5430475F002A4F58285F08312064F
:1019F300C8FFAEF0E543254075F002A42401F5824B
:101A0300E5F03400F583E0FCA3E0FDC3EF9DF54270
:101A1300EE9CF541C3E5429464E5416480948050B3
:101A23000DC3E542949CE5416480947F5026E543D1
:101A33002540FD75F002A42401F582E5F03400F59C
:101A430083EEF0A3EFF074D92DF582E43401F5832E
:101A5300E4F0805CAB3CAA3DA93EE5430475F0028B
:101A6300A4F58285F0831206C8FFAEF0E543254056
:101A7300FD75F002A42401F582E5F03400F583E05E
:101A8300FAA3E0FBC39FEA9E500F74D92DF582E4BD
:101A93003401F583E004F08017D3EB9FEA9E4010F6
:101AA300E543254024D9F582E43401F583E014F0BD
:101AB300E543254024D9F582E43401F583E0FFD3DF
:101AC30064809481500AC3EF6480947F40026189EB
:101AD300D3E5429414E54164809480500DC3E542FC
:101AE30094ECE5416480947F5022AE41AF427C0088
:101AF3007D05120651E543254075F002A42401F546
:101B030082E5F03400F583EE8FF08068AB3CAA3DAC
:101B1300A93EE5430475F002A4F58285F08312061D
:101B2300C8FFAEF0E5432540FD75F002A42401F59E
:101B330082E5F03400F583E0FAA3E0FBC39FEA9E5D
:101B4300501575F002EDA42401F582E5F03400F59B
:101B530083E475F001801DD3EB9FEA9E4019E543B2
:101B6300254075F002A42401F582E5F03400F583E5
:101B730074FFF5F0120687E543254024D9F582E486
:0A1B83003401F583E4F0054321D698
:011B8D002235
:1027D1004102A6004102A300011E00C1104202A451
:0227E100012CC9
:0301000016000DD9
:102D2D00C0D1CEBBA183674F3D2D9B19273D536667
:0A2D3D00717065554333261C1541E3
:0227E300C191A2
:04217A008E338F34DD
:10217E007B0EEB30110E3395E0FE7438240EF58293
:10218E00742D800CFF3395E0FE742D2FF582742D87
:10219E003EF583E493FF9002A1E4F0A3EFF0D39019
:1021AE0002A2E095349002A1E095334004EBFF418A
:1021BE00B81BEBFF3395E0FE30110974382FF58212
:1021CE00742D8007742D2FF582742D3EF583E493C4
:1021DE00FF9002A2E02FF09002A1E03400F09002F6
:1021EE00A1E0FEA3E0FFD39534EE9533500241B04B
:1021FE00EF9534FFEE9533FE7C007D6412063F9022
:10220E00029FEEF0A3EFF090029FE0FEA3E0FFEB43
:10221E00FD3395E0FC30110974382DF582742D8054
:10222E0007742D2DF582742D3CF583E493FD7C000F
:10223E0012065190029FEEF0A3EFF0C3EB64809470
:10224E0084EBFF40253395E0FEEF24FCFFEE34FFD8
:10225E00FE7C007D6412063F9002A0E02FF09002FB
:10226E009FE03EF0E0547FF080533395E0FE7C001B
:10227E007D6412063F9002A0E02FF090029FE03E98
:10228E00F0E0FEA3E0FFC374909FFF74019EFE90EA
:10229E00029FF0A3EFF0EE448090029FF0A3EFF0C8
:1022AE00801BEB600221BFAF03EF3395E0FE7C0095
:1022BE007D6412063F90029FEEF0A3EFF090029F16
:0522CE00E0FEA3E0FFAB
:0122D30022E8
:10200000900298EFF0A3ECF0A3EDF0A3EAF0A3EBBD
:10201000F0EF701E90029BE0FEA3E0FF90029AE0BA
:102020002FFF900299E03ECF2480CF34FF90029D95
:10203000216D900298E0FF64016005EF6402707CFE
:10204000900299E0FEA3E0FF12217A900296EEF052
:10205000A3EFF0EE90029630E712E0547FFEA3E08B
:10206000FFC3E49FFFE49E90029D8008E0FFA3E091
:1020700090029DCFF0A3EFF0900298E0B40222907E
:10208000029DE0FEA3E0FF7C007D0912063F7D0576
:10209000120651EF2440FFEE340190029DF0A3EFB1
:1020A000F090029BE0FEA3E0FF90029EE02FFF90E5
:1020B000029DE03ECF2480CF34FF216D900298E056
:1020C000B40328A3E0FCA3E0FDEC1204377B007A04
:1020D000C0797F7844120395E4FBFA79C8784212FC
:1020E000028C12047090029DEE216D900298E0FF28
:1020F00064046005EF64057078900299E0FCA3E049
:10210000FDEC1204377B007AC0797F784412039586
:10211000E4FBFA7948784212028C1204709002961D
:10212000EEF0A3EFF0D39418EE648094805012A3E5
:10213000E0FFB40504D212802BEFB40427C2128052
:1021400023C3900297E0941A900296E064809480F2
:102150004012900298E0FFB40504C2128006EFB46A
:102160000402D212A212E4FF3390029DCFF0A3EF3B
:09217000F090029DE0FEA3E0FFE7
:012179002243
:1027E5004402920200020048028A006800690066FD
:0927F500006744028600020002A4
:0E2C6A00853683E49390029DFFF0AC38AD39BF
:102C7800AB07C2AF75F65575F6AA75F65543BF048E
:0E2C88008CF48DF58BF675F780D2AF7F0022AD
:102D1100C2AF75F65575F6AA75F65543BF04EF2592
:0C2D2100E0F5F4E4F5F575F782D2AF227E
:0B2DB7008F828E83E49312062D7F01B3
:012DC20022EE
:0C2CB700E52675F002A42448F9E4FAFBBD
:102CC30012069DF58285F083E4932402FFE4338F9B
:042CD300F002070004
:022B5A00A907C9
:102B5C00E925E02486F582E43402F583A3E0F5351B
:102B6C00E925E02448F8E6FE08E6FFE5352402FDF9
:102B7C00E433FCE925E0244CF8E6FA08E6C39DFDB5
:0D2B8C00EA9CFCC3EF9DEE9C4002D322C3E7
:012B99002219
:102D9300E4F525AF251210000525E525C39402406F
:012DA300F23D
:012DA400220C
:021000008F2639
:10100200EF25E02492F582E43402F583E0F529A38A
:10101200E0F52AEF25E025E0248AF582E43402F5A2
:1010220083A3E0F527EF25E025E0248CF582E43464
:1010320002F583A3E0F528E52725E0F52B752C00C2
:10104200E52825E0752DFFF52E752F00852C82856C
:101052002B83E4936455600221A6AB2DAA2EA92FFF
:101062001205E76455600221A6E52C2401FFE43550
:101072002BFEE52625E02448F8A60608A607E52665
:1010820025E02448F8E6FE08E6F5828E83E493F430
:101092006020E52625E02448F8E6FE08E6AA06C315
:1010A200852E83852F829582EA95835005122CB76F
:1010B20080CCE52625E02448F8E6FE08E6C3952C18
:1010C200F531EE952BF530E52F2401F9E4352EFEAE
:1010D200AF01E52625E02448F8A60608A607E5267E
:1010E20025E02448F8E6FE08E6F5828E83E493F4D0
:1010F2006030AB2DE52F252AF9E52E3529FAC003FC
:101102008A838982E52625E02448F8E6FE08E6AAD5
:1011120006F9C3D0E0E99582EA95835005122CB70F
:1011220080BCE52625E02448F8E6FE08E6AB2DAAB9
:101132002EA92FAC02AD01C39DFFEE9CFED3EF950D
:1011420031EE95305032AE02AF01EF2401FFE43EA2
:10115200FEE52625E02444F8A60608A607745025D5
:1011620026F8A627AE2BAF2CAD07AC06E4FF122C57
:1011720078EF70024127C322E52C2401FFE4352BCE
:10118200FEE52625E02444F8A60608A607745025A5
:1011920026F8A628AC2EAD2FE4FF122C78EF7002B1
:1011A2004127C322852C82852B83E493B4551EE507
:1011B2002C2401FFE4352BFEE52625E02444F8A685
:1011C2000608A60774502526F8A6288058AB2DAA33
:1011D2002EA92F1205E7B45520AE02AF01EF24016C
:1011E200FFE43EFEE52625E02444F8A60608A6070D
:1011F20074502526F8A627802CAE2BAF2CAD07AC59
:1012020006ED2401FFE43CFEE52625E02444F8A691
:101212000608A60774502526F8A6287F55122C78B2
:10122200EF6002C322E52625E02444F8E6FE08E644
:10123200FFE52625E02448F8A60608A607E52625A8
:10124200E02444F8E6FE08E6252AFFE5293EFEE50D
:101252002625E0244CF8A60608A607E52625E02464
:1012620048F8E6FE08E6F5828E83E493F460051200
:051272002CB780E7D35A
:011277002254
:021800008F3522
:10180200EF25E02444F8E6FE08E68E36F5377450FC
:101812002FF8E625E0F538753900E53525E0249204
:10182200F582E43402F583E0FFA3E090029ECFF05C
:10183200A3EFF0E490029AF0E53525E02492F582D8
:10184200E43402F583E0C313FF90029AE0C39FE4FD
:1018520094005015122DE274502535F8E6FFE02F62
:10186200FF122D11E004F080CF90029FE02537FF98
:1018720090029EE03536CF24FFF53BEF34FFF53A78
:101882000539E53970020538853782853683E49358
:10189200F470022130C3E537953BE536953A4002B4
:1018A2002130122DE2853782853683740193FF60E1
:1018B20072F4606FE49390029B122C72EF60037FCC
:1018C20001220539E539700205380537E53770021E
:1018D2000536F582122C6AEF60037F01220539E595
:1018E20039700205380537E53770020536E4900293
:1018F2009AF090029BE0FF90029AE0C39F50898584
:101902003782122C6AEF60037F01220539E53970B4
:101912000205380537E5377002053690029AE00471
:10192200F080CF7B007A007936122CC3018AE5352C
:1019320025E02448F8A63808A639E53525E02444F0
:10194200F8E6FEEEC31390029CF0FD74502535F8C4
:10195200E625E0FEE53525E02444F8A606087600F3
:1019620074502535F8A605E53525E02444F8E6FE51
:1019720008E6FF90029FE02FFF90029EE03EFEE508
:101982003525E0244CF8A60608A607E53525E0240F
:1019920044F8E6FC08E6FD7F55122C78EF60037FE1
:1019A200012274502535F8E67D0025E0FCE4FF12A3
:1019B2002C78EF60037F0122E53525E02444F80806
:0819C20006E6187001067F0023
:0119CA0022FA
:0816B2008F358B368A37893829
:1016BA00E4F53DF53EE53925E02486F582E4340279
:1016CA00F583A3E0F53FE53925E02444F8E6FE0872
:1016DA00E68E3AF53B0535E53925E02448F8E6FE7D
:1016EA0008E6FFE53F2401FDE433FCE53925E02463
:1016FA004CF8E6FA08E6C39DFDEA9CFCD3EF9DEEA2
:10170A009C400122853B82853A83740193FE6535AC
:10171A006010E493F4600B7B007A00793A122CC3D0
:10172A0080E2EEB5350BE53B2401F53EE4353AF5AA
:10173A003DE53925E02448F8E6FE08E6FDAC06AFAB
:10174A003F122C78EF6002C322E53925E02448F8DD
:10175A0008740226F618E436F6E4F53CE53CC3952F
:10176A003F5030E53925E02448F8E6FE08E6253CF6
:10177A00FFE43EFEAD07FCAB36AA37A938853C82AA
:10178A00758300120600FF122C78EF6002C322054F
:10179A003C80C9AF3F7E00E53925E02448F808EFD0
:1017AA0026F618EE36F6E53925E02448F8E6FC0870
:1017BA00E6FDEF2401FFEE33FEC3ED9FFFEC9EFE34
:1017CA00AD07FCAF35122C78EF6002C322E53E4527
:1017DA003D6012AE3DAF3EAD07AC06E4FF122C7879
:0617EA00EF6002C322D3F0
:0117F00022D6
:0825A0008F2E8B2F8A30893148
:1025A800E53225E02444F8E6FE08E68E33F534E407
:1025B800F535F536052E853482853383E493F4604A
:1025C80049E53225E0244CF8E6FC08E6FDC3E5348D
:1025D8009DE5339C5034740193652E7022E5364591
:1025E800356016E5362401FFE43535FEAD07FCE419
:1025F800FF122C78EF6002C3228533358534367B91
:10260800007A007933122CC380ACE5364535603D3D
:10261800853682853583740293FFAB2FAA30A931A2
:10262800E48FF0120738AB2FAA30A93112069D7536
:10263800F000120738853682853583740393FFAB23
:0E2648002FAA30A931E48FF0120700D322C36D
:012656002261
:0826FA008F2F8B308A318932E9
:10270200E53325E02444F8E6FE08E68E34F535E4A8
:10271200F536F537052F853582853483E493F460E9
:1027220049E53325E0244CF8E6FC08E6FDC3E5352F
:102732009DE5349C5034740193652F7022E5374532
:10274200366016E5372401FFE43536FEAD07FCE4BA
:10275200FF122C78EF6002C3228534368535377B31
:10276200007A007934122CC380ACE5374536601408
:10277200853782853683740393AB30AA31A932122E
:05278200062DD322C367
:01278700222F
:0428FB008F2F8B3060
:1028FF00E4F531EDF533ECF532122DE2AF30122B5A
:10290F005A5022E531C3940A500CAF30121800EF21
:10291F006004053180ED7F057E001217F5E531C3A8
:10292F00940A400122E531C3940A50147B007A00C7
:10293F007932853039AF2F1216B24004053180E558
:09294F00E531C3940A400122D3D2
:01295800225C
:10028C00EC4D6011E8497017ED33EC3304600DE46C
:10029C00FCFFFEFD22E933E8330470F80204DC12A3
:1002AC0004A758046009E4CC2481500628500902A4
:1002BC0004E62840030204E3C0E0EB4A7044B98032
:1002CC0006D0E0FB0204D2EF4E701CBD8008EBFFA1
:1002DC00EAFEE9FD80EBE98DF0A4FEE5F002037582
:1002EC00E9CDF9EAFEEBFFEF89F0A4FCE5F0CE894D
:1002FC00F0A42EFFE435F0CD89F0A42DFEE435F00A
:10030C008067EF4E7005BD80D780C3EF8BF0A4AC37
:10031C00F0EE8BF0A42CFCE435F0F8EF8AF0A42C72
:10032C00E5F038FCE433CB8DF0A42CFCE5F03BF885
:10033C00EE8AF0A42CFCE5F038F8E433CF89F0A475
:10034C002CFCE5F038CF3400CE89F0A42FFFE5F07B
:10035C003EFEE433C98DF0A42EFEE5F039CD8AF0D3
:10036C00A42FFFE5F03EFEE43DFD33D0E0FB50074B
:10037C000BBB000F0204E6EC2CFCEF33FFEE33FE5C
:06038C00ED33FD0204BE8A
:100392000204E6EC5D046005E8590470030204DC23
:1003A2001204A7580460F6EC4860F2EC7004FDFEFB
:1003B200FF22C860DB2481C85009C398600250063E
:1003C2000204E39850CAF582E9294B4A7005AB82D0
:1003D2000204D275F0007C1A7880C3EF9BEE9AED8E
:1003E20099400DC3EF9BFFEE9AFEED99FDE842F0B6
:1003F200DC23ACF0D0E0FFD0E0FED0E0FDAB822009
:10040200E7101BEB60BAEC2CFCEF33FFEE33FEED92
:1004120033FD0204BEE803F830E705C0F075F000D2
:10042200EF2FFFEE33FEED33FD40B830E7C280AA76
:1004320075F020800E75F010800575F0087D007E45
:10044200007F003392D530D503120874EC3340108C
:10045200EF33FFEE33FEED33FDEC33FCD5F0ED224E
:0E046200E5F0247EA2D513CC92E7CDCEFF228A
:10047000EDD2E7CD33EC3392D524814006E4FFFE84
:10048000FDFC22FCE4CFCECDCC24E0501174FF80E3
:10049000EDC3CC13CCCD13CDCE13CECF13CF047080
:0704A000F030D5DE02087404
:1004A700E9D2E7C933E833F892D5EDD2E7CD33EC9B
:0704B70033FC5002B2D52214
:1004BE00EC30E7100FBF000C0EBE00080DBD00049F
:1004CE000BEB6014A2D5EB13FCED92E7FD2274FF4B
:1004DE00FCFDFEFF22E480F8A2D574FF13FC7D80A4
:0304EE00E480EFB8
:03000000020200F9
:0C020000787FE4F6D8FD7581BA02024751
:1004F100E709F608DFFA8046E709F208DFFA803EED
:1005010088828C83E709F0A3DFFA8032E309F608D9
:10051100DFFA8078E309F208DFFA807088828C8341
:10052100E309F0A3DFFA806489828A83E0A3F608F5
:10053100DFFA805889828A83E0A3F208DFFA804CCF
:1005410080D280FA80C680D4806980F280338010A6
:1005510080A680EA809A80A880DA80E280CA80330F
:1005610089828A83ECFAE493A3C8C582C8CCC58387
:10057100CCF0A3C8C582C8CCC583CCDFE9DEE78057
:100581000D89828A83E493A3F608DFF9ECFAA9F0D6
:10059100EDFB2289828A83ECFAE0A3C8C582C8CC2C
:1005A100C583CCF0A3C8C582C8CCC583CCDFEADE45
:1005B100E880DB89828A83E493A3F208DFF980CCA7
:1005C10088F0EF60010E4E60C388F0ED2402B404A0
:1005D1000050B9F582EB2402B4040050AF23234547
:0605E10082239005417326
:1005E700BB010689828A83E0225002E722BBFE0212
:0905F700E32289828A83E4932245
:10060000BB010CE58229F582E5833AF583E02250AF
:1006100006E92582F8E622BBFE06E92582F8E222F9
:0D062000E58229F582E5833AF583E4932213
:10062D00BB010689828A83F0225002F722BBFE01AC
:02063D00F322A6
:10063F00EF8DF0A4A8F0CF8CF0A428CE8DF0A42ECF
:02064F00FE2289
:10065100C2D5EC30E709B2D5E4C39DFDE49CFCEEC4
:1006610030E715B2D5E4C39FFFE49EFE120898C39C
:10067100E49DFDE49CFC800312089830D507C3E497
:060681009FFFE49EFE2233
:10068700C5F0F8A3E028F0C5F0F8E58215827002FE
:060697001583E038F0229B
:10069D00BB010A89828A83E0F5F0A3E02250068728
:1006AD00F009E71922BBFE07E3F5F009E3192289EA
:0B06BD00828A83E493F5F0740193221D
:1006C800BB0110E58229F582E5833AF583E0F5F070
:1006D800A3E0225009E92582F886F008E622BBFE4D
:1006E8000AE92582F8E2F5F008E222E5832AF58393
:0806F800E993F5F0A3E9932258
:10070000BB010789828A83020687500B09C5F0273F
:10071000F7C5F01937F722BBFE0D09F8E325F0F312
:10072000C5F019E338F322F889828A83740193258E
:08073000F0C5F0F8E493382253
:10073800BB010A89828A83F0E5F0A3F0225006F70C
:0F07480009A7F01922BBFE06F3E5F009F3192209
:10075700E88FF0A4CC8BF0A42CFCE98EF0A42CFC41
:100767008AF0EDA42CFCEA8EF0A4CDA8F08BF0A4BF
:100777002DCC3825F0FDE98FF0A42CCD35F0FCEB1E
:100787008EF0A4FEA9F0EB8FF0A4CFC5F02ECD39E3
:0F079700FEE43CFCEAA42DCE35F0FDE43CFC2250
:1007A60075F008758200EF2FFFEE33FECD33CDCC0A
:1007B60033CCC58233C5829BED9AEC99E58298408D
:1007C6000CF582EE9BFEED9AFDEC99FC0FD5F0D66A
:1007D600E4CEFBE4CDFAE4CCF9A88222B800C1B994
:1007E6000059BA002DEC8BF084CFCECDFCE5F0CBD2
:1007F600F97818EF2FFFEE33FEED33FDEC33FCEB0B
:1008060033FB10D703994004EB99FB0FD8E5E4F9C5
:10081600FA227818EF2FFFEE33FEED33FDEC33FCB2
:10082600C933C910D7059BE99A4007EC9BFCE99AA6
:10083600F90FD8E0E4C9FAE4CCFB2275F010EF2FEB
:10084600FFEE33FEED33FDCC33CCC833C810D707EB
:100856009BEC9AE899400AED9BFDEC9AFCE899F826
:0E0866000FD5F0DAE4CDFBE4CCFAE4C8F922B9
:0E087400C3E49FFFE49EFEE49DFDE49CFC2295
:10088200EB9FF5F0EA9E42F0E99D42F0EC6480C8ED
:0608920064809845F0228D
:102B1900AC63AD64AE65AF66780FEFA2E2EC20E678
:102B290001B35D5E5FF47004FCFDFEFFEF13FFEE81
:102B390013FEED13FDEC13FCD8E08C638D648E65F8
:102B49008F66EE547FFE228E638F64E4F565F56629
:012B59002259
:102DA500C3EE6480948040028007C3E49FFFE49EE5
:022DB500FE22FC
:10020C00021EADE493A3F8E493A34003F68001F23D
:10021C0008DFF48029E493A3F85407240CC8C333F3
:10022C00C4540F4420C8834004F456800146F6DFC2
:10023C00E4800B0102040810204080902788E47EA3
:10024C00019360BCA3FF543F30E509541FFEE493B7
:10025C00A360010ECF54C025E060A840B8E493A37E
:10026C00FAE493A3F8E493A3C8C582C8CAC583CAA9
:10027C00F0A3C8C582C8CAC583CADFE9DEE780BE61
:0127FE0000DA
:10089800BC000BBE0029EF8DF084FFADF022E4CC44
:1008A800F875F008EF2FFFEE33FEEC33FCEE9DEC0D
:1008B800984005FCEE9DFE0FD5F0E9E4CEFD22ED53
:1008C800F8F5F0EE8420D21CFEADF075F008EF2F9D
:1008D800FFED33FD4007985006D5F0F222C398FD8E
:0508E8000FD5F0EA222B
:00000001FF
